:020000040800F2
:100000000080012081240008D1240008D1240008A8
:10001000D1240008D1240008D124000800000000E9
:10002000000000000000000000000000D1240008D3
:10003000D124000800000000D12400082B21000872
:10004000D1240008D1240008D1240008D1240008BC
:10005000D1240008D1240008952100089B21000824
:10006000A1210008A7210008AD210008D124000823
:10007000D1240008D1240008D1240008D12400088C
:10008000D1240008D1240008D12400080000000079
:10009000000000000000000000000000B321000884
:1000A00051260008F125000861260008D124000827
:1000B0001126000821260008312600081D27000807
:1000C000292700083527000841270008D124000807
:1000D000D1240008A1280008B92800080000000069
:1000E000C921000875240008D12400080000000080
:1000F000000000000000000000000000D124000803
:1001000000000000D124000841260008D124000886
:1001100000000000000000000000000000000000DF
:10012000D1240008D1240008D1240008D1240008DB
:10013000D1240008000000000000000000000000C2
:10014000000000000000000000000000D1240008B2
:10015000D1240008D1240008D1240008D1280008A7
:100160004D2700085927000800000000000000008B
:10017000000000000000000000000000000000007F
:1001800000000000D1240008000000000000000072
:04019000D12400086E
:1001940010B5054C237833B9044B13B10448AFF3BD
:1001A40000800123237010BD2800002000000000FF
:1001B400702A00080C4B43B10C480D4910B5AFF33D
:1001C40000800C48036823B910BD0A48036833B99A
:1001D4007047094B002BF7D0BDE810401847064B79
:1001E400002BF5D0184700BF00000000702A00085B
:1001F4002C000020280000200000000053B94AB958
:10020400002908BF00281CBF4FF0FF314FF0FF301A
:1002140000F07AB9ADF1080C6DE904CE00F006F8EF
:10022400DDF804E0DDE9022304B070472DE9F0476E
:100234008C460D460446089E002B51D18A4217462F
:100244006DD9B2FA82FEBEF1000F0BD0CEF1200CB4
:1002540001FA0EF520FA0CFC02FA0EF74CEA050C32
:1002640000FA0EF44FEA174A250CBCFBFAF81FFA01
:1002740087F90AFB18CC45EA0C4508FB09F3AB42A5
:100284000AD9ED1908F1FF3280F02381AB4240F224
:100294002081A8F102083D44ED1AA4B2B5FBFAF09E
:1002A4000AFB105544EA054400FB09F9A14509D9A4
:1002B400E41900F1FF3380F00A81A14540F207817F
:1002C40002383C44A4EB090440EA08400021002E13
:1002D40061D024FA0EF4002334607360BDE8F08723
:1002E4008B4207D9002E54D0002186E8210008460D
:1002F400BDE8F087B3FA83F1002940F08E80AB4269
:1003040002D3824200F2FA80841A65EB03050120CD
:10031400AC46002E3FD086E81010BDE8F08712B935
:100324000127B7FBF2F7B7FA87FEBEF1000F34D10D
:10033400EB1B3A0C1FFA87FC0121B3FBF2F8250CE6
:1003440002FB183345EA03450CFB08F3AB4207D91B
:10035400ED1908F1FF3002D2AB4200F2D1808046A1
:10036400ED1AA3B2B5FBF2F002FB105543EA0544C3
:100374000CFB00FCA44507D9E41900F1FF3302D2B9
:10038400A44500F2B8801846A4EB0C0440EA0840E7
:100394009DE731463046BDE8F087CEF1200405FAEA
:1003A4000EF307FA0EF720FA04F83A0C25FA04F4CF
:1003B40048EA0308B4FBF2F14FEA184502FB114482
:1003C4001FFA87FC45EA044501FB0CF3AB4200FA33
:1003D4000EF409D9ED1901F1FF3080F08A80AB42A7
:1003E40040F2878002393D44EB1A1FFA88F5B3FBCB
:1003F400F2F002FB103345EA034500FB0CF3AB4279
:1004040007D9ED1900F1FF386FD2AB426DD902382C
:100414003D44EB1A40EA01418FE7C1F1200722FA7B
:1004240007F88B4005FA01F448EA030320FA07FEB3
:100434004FEA134CFD404EEA040EB5FBFCF94FEABB
:100444001E440CFB19551FFA83F844EA054509FBC1
:1004540008F4AC4202FA01F200FA01FA08D9ED18E4
:1004640009F1FF3043D2AC4241D9A9F102091D443C
:100474002D1B1FFA8EFEB5FBFCF00CFB10554EEA4B
:10048400054400FB08F8A04507D9E41800F1FF353E
:1004940029D2A04527D902381C4440EA0940A4EBDC
:1004A4000804A0FB02894C45C6464D4615D312D01C
:1004B40056B1BAEB0E0364EB050404FA07F7CB401C
:1004C4001F43CC40376074600021BDE8F0871846B4
:1004D400F8E69046E0E6C245EAD2B8EB020E69EBD4
:1004E40003050138E4E72846D7E7404691E781460B
:1004F400BEE7014678E702383C4445E7084608E78A
:10050400A8F102083D442BE7704700BF01211720E2
:1005140002F0E8B908B50121172002F037FA4FF4C8
:100524007A7002F055FA1720002102F02FFA4FF4E6
:100534007A70BDE8084002F04BBA000000B53022E2
:1005440099B000210DEB020002F088FA1422002178
:1005540002A802F083FA1422002107A802F07EFA0E
:100564002A4B002100911A6C42F080521A641B6CD1
:10057400274A03F080530093009B0191136823F4EE
:10058400404343F400431360136803F4404301936E
:10059400019B0B2310220C934FF480330D93109284
:1005A40001234FF480020F93119313920223042228
:1005B400129314921693482203230CA815921793AE
:1005C40000F0AEFF18B19521124801F080FF002120
:1005D4000F2302A80293039104910591069101F05F
:1005E4004FF918B1A2210B4801F071FF02230793C0
:1005F40007A84FF400730A9301F0DCF918B1A8219D
:10060400044801F064FF19B05DF804FB00380240AF
:1006140000700040382C0008B0F86A30013303F051
:100624003F03A0F86A30B0F86A30B0F868009BB2B3
:1006340098424FF0FF3018BF00207047B0F8F430F4
:10064400B0F8F600181A00F03F007047B0F8F43024
:10065400B0F8F6209BB293421ABFD0F8F030985C01
:100664004FF0FF307047B0F8F420B0F8F63092B293
:100674009A421FBFD0F8F020D25C013303F03F034D
:100684001ABFA0F8F63010464FF0FF307047000054
:1006940010B5B0F8FC4001230374E31803F03F03E2
:1006A400B0F8FE2092B29342FAD0D0F8F820115557
:1006B40000F19404A0F8FC30204602F051F818B977
:1006C4000249204602F05EF8012010BD1D06000814
:1006D400037C33B1B0F8FC20B0F8FE309BB29A42F0
:1006E400FAD1704700F11103C0F8F03000F1510263
:1006F4000023A0F8F430A0F8F630C0F8F820A0F8F1
:10070400FC30A0F8FE30704738B5002343604FF446
:100714007A7383600F4B03600F4B984204460D4677
:100724000BD10E4B1A785B7880F8ED2080F8EC3012
:100734002046FFF7D7FF204638BD0949284601F077
:1007440073FE084984F8ED00284601F06DFE84F834
:10075400EC00EDE7D42C000844000020912C0008A4
:10076400F02B0008142C000801490248FFF7CCBF05
:1007740000440040440000202DE9F04106460D46A7
:1007840001EB02080C464445A4EB050707D0336887
:1007940014F8011B1B68304698470028F3D13846EB
:1007A400BDE8F08110B5044602F010F9E06023685A
:1007B4002046DB689847002808DA02F007F9E36866
:1007C400C01AA3689842F2D34FF0FF3010BD2DE950
:1007D400F04180460D468F180C46BC42A4EB05063A
:1007E40007D04046FFF7DEFF002802DB04F8010BC8
:1007F400F3E73046BDE8F0812DE9F84380468946A9
:1008040016461C467BB1D7181546AF42A5EB060425
:1008140009D04046FFF7C6FF002804DB484502D054
:1008240005F8010BF1E72046BDE8F883836810B5AD
:10083400044613B1032201469847204610BD000028
:1008440008B5044B2BB10448FFF7F8FE08B1AFF329
:10085400008008BD000000004400002001F06BBCD3
:100864007047704708B5032000F066F8BDE80840FB
:10087400FFF7F4BF08B5FFF7F4FFFFF747FE044C9A
:10088400FFF748FE002CFBD0FFF7DAFFF8E700BFC4
:10089400450800087047000038B50E4A0E4B05465F
:1008A40018784FF47A73B3FBF0F31068B0FBF3F0ED
:1008B40000F096F8044658B90F2D09D80246294687
:1008C4004FF0FF3000F04AF8044B20461D6038BD5D
:1008D400012038BD2400002004000020080000206E
:1008E40008B50B4B1A6842F400721A601A6842F495
:1008F40080621A601A6842F480721A60032000F061
:100904001BF80020FFF7C8FFFFF7C4FF002008BD55
:10091400003C0240034A044B11681B780B441360EB
:10092400704700BF0C04002004000020014B18682D
:10093400704700BF0C040020074AD36823F4E06327
:100944001B041B0C43F0BF63000243F4003300F4A8
:10095400E0600343D360704700ED00E0174B30B50F
:10096400DC68C4F30224C4F10703251D042B28BF4B
:100974000423062D4FF0010505FA03F303F1FF33B9
:100984008CBF033C00241940A14005FA04F4013C47
:100994002240002842EA01024FEA0212ADBF00F1F0
:1009A400604000F00F00064B00F56140B5BFD2B2C5
:1009B400D2B21A5480F8002330BD00BF00ED00E02D
:1009C40014ED00E0002808DB4209012300F01F00B9
:1009D40003FA00F0014B43F82200704700E100E005
:1009E4000138B0F1807F0AD2064B074A5860F021E3
:1009F40082F823100020072298601A6070470120B3
:100A0400704700BF10E000E000ED00E0002809DBC3
:100A14004309012200F01F0002FA00F06033024A89
:100A240042F82300704700BF00E100E0704708B5BA
:100A3400FFF7FCFF08BD90F83530022B03D080236C
:100A44004365012070470268052380F83530136838
:100A540023F00103136000207047000008B5044B25
:100A64005969014202D0586101F07CFB08BD00BF06
:100A7400003C014037B590F83D40282C34D1002982
:100A840030D0002A2ED090F83C40012C2CD00568A0
:100A9400012480F83C402C68E4075EBF2C6844F0D5
:100AA40001042C602C6824F400642C60292480F850
:100AB4003D40202480F83E40002404644285C36203
:100AC400438D019403856B690193AB690193019B89
:100AD4006B68416243F4E06380F83C406B602046FD
:100AE40003B030BD0120FBE70220F9E737B590F8E9
:100AF4003D40282C34D1002930D0002A2ED090F843
:100B04003C40012C2CD00568012480F83C402C6822
:100B1400E4075EBF2C6844F001042C602C6824F4C4
:100B240000642C602A2480F83D40202480F83E4054
:100B3400002404644285C362438D019403856B6978
:100B44000193AB690193019B6B68416243F4E063D9
:100B540080F83C406B60204603B030BD0120FBE7C9
:100B64000220F9E790F83D30202B14D1282380F897
:100B74003D3003681A68D2075EBF1A6842F001026A
:100B84001A601A6842F480621A605A6842F4407229
:100B94005A600020704702207047704770477047C2
:100BA4007047704790F83D30293B012B10B503681E
:100BB400044639D800220263282280F83D201A68AE
:100BC40022F400621A605A6812F4006254D05A681F
:100BD400606B22F400625A6090F83530012B394B77
:100BE40031D00365FFF727FF50B12268606B1368AB
:100BF40023F001031360202384F83D30036D9847EC
:100C040094F83D30282B0ED1236C5B070BD52E4B6B
:100C1400E362202200232363204684F83D2084F8E5
:100C24003E3001F046FD10BD90F83D20602A05D00D
:100C34005A6812055CBF202280F83D2000222263FE
:100C440084F83E20BBE7A06B0365FFF7F4FE0028A1
:100C5400D6D022685369580604D5636A1269591CB0
:100C640061621A702268A06B136823F00103136099
:100C7400202384F83D30C1E794F83D10602914D155
:100C8400202184F83D1022645A69510604D5626A11
:100C94001B69511C616213702268136823F00103FD
:100CA40013602046FFF77DFFAAE75A69520604D570
:100CB400626A1B69511C61621370204601F026FDB3
:100CC4009EE700BFD91400080000FFFF0368F0B5D9
:100CD4009D6959695A6890F83E40E4B2102C8DB071
:100CE40002D0402C40F0558211F0011F66D09705C8
:100CF40064D590F83E40402C43D1046D002C3BD188
:100D0400446C04F0FE041C61984E994C2E400C4037
:100D1400002E00F09F81974D0D40002D00F066815C
:100D2400550540F16381002C40F0608190F83D202E
:100D3400058D90F83E10C46AD2B2C9B2002D40F0BD
:100D44000581212A40F00481042C00F06C81082CD8
:100D540000F0698114F5803F00F065815A6822F43F
:100D6400E0625A601123036380F83E50202380F828
:100D74003D30FFF712FFF6E0446C44F00104E4B2A6
:100D8400C1E70469B4F5804F05D190F83D40212CAA
:100D9400446CF2D1B5E7046D34B9446CE41104F049
:100DA400060444F0F004AEE7046D012CACD1446CAD
:100DB400E41104F0060444F0F104A4E76E4C0C4082
:100DC4001CB1960501D5446CD9E76C4C0C40002C41
:100DD4009AD0940598D590F83E40C66AD0F830E091
:100DE40090F83D70222FE4B240F0A880076D47B917
:100DF400402C06D101975C6901949C690194019C83
:100E040082E7046D8CB90769B7F5404F0DD10294A0
:100E14005C6902949C690294029C1C6844F480748A
:100E24001C60046D013404656EE7448DA4B254B9AA
:100E340003945C6903949C690394039C1C6844F4C4
:100E440000741C6019E0448DA4B2012C42D116F543
:100E5400803F1BD11C6824F480641C605C6814F41B
:100E640000640CD01C6824F480641C600024049486
:100E74005C6904949C690494049C0024D3E705945D
:100E84005C6905949C690594059CD7E7042E15D0EC
:100E9400082E13D0BEF1120F10D0C46A022C1C68A5
:100EA40014BF24F4806444F480641C600024069419
:100EB4005C6906949C690694069CDEE71C6824F42D
:100EC40080641C60002407945C6907949C690794FF
:100ED400079CB3E7448DA4B2022C1CD1C46A022C33
:100EE4001C681DBF24F480641C601C6844F4806486
:100EF40018BF44F400641C605C68270542BF5C684A
:100F040044F480545C60002408945C6908949C69EF
:100F14000894089CB1E71C6844F480641C605C6815
:100F2400260542BF5C6844F480545C600024099444
:100F34005C6909949C690994099C9EE700240A94BD
:100F44005C690A949C690A940A9CDDE6212A03D010
:100F5400402908D1222A06D1428D92B282B95A6818
:100F640022F480625A600DB0F0BD00BF040010008E
:100F740004000100800001000800010002000100DB
:100F840090F83E20402A27D1026D7AB9C26C012A1A
:100F9400826C05D1D2B21A61036D02330365E2E7B4
:100FA400C2F307221A61036D0133F7E7026D012AC8
:100FB40002D1826CD2B2F5E7026D022AD3D190F845
:100FC4003D20222A04D11A6842F480721A60CAE7CA
:100FD40090F83D20212AC6D1426A511C4162127800
:100FE4001A61438D013B9BB24385BCE7002CBAD008
:100FF4009405B8D5C16A90F83D20212AB3D1428D19
:1010040092B2002AE8D104290DD008290BD011F599
:10101400803F08D0596821F4E061596011230363CB
:1010240080F83E20A2E65A6822F4E0625A601A6808
:1010340042F400721A6000232022036380F83D20EA
:1010440090F83E2080F83E30402A7FF492AEFFF7BD
:10105400A6FD88E7904D0D40002D41D051053FD5A8
:10106400002C3DD190F83D20222A7FF47CAF428DA4
:1010740092B2032A13D9426A1B69511C416213704C
:10108400438D013B9BB24385438D9BB2032B7FF47D
:101094006AAF0268536823F48063536063E7012AEC
:1010A4003FF661AF1A6822F480621A605A6822F42B
:1010B400E0625A60426A1B69511C41621370438D9D
:1010C400013B9BB24385202380F83D30046390F8B4
:1010D4003E3080F83E40402B58D1FFF761FD42E797
:1010E400002C3FF440AF97057FF53DAFC16A428DB8
:1010F40092B2042A426A08D1596821F48061596085
:10110400511C1B69416213706BE7448DA4B2032C1C
:1011140008D1596821F480615960196821F480610B
:101124001960EDE7448DA4B2022CE9D101390129FB
:1011340019689DBF21F480611960196841F4007138
:1011440098BF41F4807119601B69511C416213708E
:10115400438D013B9BB24385436A5A1C4262026839
:1011640012691A70438D0268013B9BB24385536830
:1011740023F440735360202380F83D30002303633D
:1011840090F83E2080F83E30402AA5E7FFF706FDA0
:10119400E9E6424C0C4074B196050CD599699B69FB
:1011A40081F004011D06C1F3800154BF8289028BC2
:1011B40001F05CFAD7E63A4C0C40002C74D094054C
:1011C40072D590F83D20596821F4E06159600021FE
:1011D4000B9159690B91196841F0010119600B9940
:1011E400196821F48061196059680905D2B20CD5D7
:1011F40090F83D10222903D090F83D102A2929D1D6
:10120400816B0968496889B24185418D89B2E1B130
:1012140059694F0708D5416A1B694C1C44620B701D
:10122400438D013B9BB2438501684B695E0608D53B
:10123400436A09695C1C44621970438D013B9BB28B
:101244004385036C43F004030364036C23B1FFF789
:10125400A9FC88E6416BD4E7A2F1280102290AD847
:10126400104AC2622022036380F83D2080F83E3099
:1012740001F01FFA77E6036B222B02D0222A7FF4B7
:1012840072AE00232022036380F83D2080F83E30B4
:1012940001F026FA67E600BF4000010002000100E9
:1012A400100001000000FFFF394E3A4C2E400C4064
:1012B400002E36D0384D0D403DB3550525D524BB01
:1012C40090F83D10428D92B2C9B2002A3FF44BAE61
:1012D400426A541C446212781A61428D013A92B2F5
:1012E4004285428D92B2002A7FF43DAE29297FF4D3
:1012F4003AAE5A6822F480625A6021230363282399
:1013040080F83D3001F0FEF92DE6002C3FF42BAEC1
:1013140094057FF528AE428D92B2002A7FF45CAE2C
:1013240021E61E4D0D4035B3510524D51CBB90F864
:101334003D20418D89B2D2B200293FF414AE416AF6
:101344001B694C1C44620B70438D013B9BB243856B
:10135400438D9BB2002B7FF406AE2A2A7FF403AEA2
:101364000268536823F480635360222303632823B1
:1013740080F83D308CE7002C3FF4F5AD92057FF505
:10138400F2AD428D92B2002A3FF4EDAD426AB7E667
:10139400040010000400010080000100400001006E
:1013A400F8B50368494A5E695D681642044608D088
:1013B400E80506D5226C42F0010222646FF48072C3
:1013C4005A6116F4813F08D0E90506D5226C42F033
:1013D400020222646FF400725A6116F4823F36D01E
:1013E400EA0534D594F83E70618D94F83D20206B65
:1013F400202F89B2D2B258D1002956D102F0F70178
:10140400212903D0282A50D121284ED194F83D20F7
:10141400E16A0429D2B201D008292CD1282A2AD180
:101424002B4AE2625A6822F4E0625A606FF48062E6
:101434005A611A6822F480621A600023202223630E
:10144400204684F83D2084F83E3001F032F916F449
:10145400843F09D0EB0507D5236C43F008032364CC
:1014640023686FF400625A61236C73B32046BDE8AD
:10147400F840FFF797BB212A23D11549E162226383
:10148400202284F83D20002284F83E205A6822F469
:10149400E0625A606FF480625A611A6822F48062D2
:1014A4001A60204601F02EF9D1E7226C42F00402C2
:1014B400226494F83E20102A02BF1A6842F4007293
:1014C4001A606FF480625A61C1E7F8BD000101003F
:1014D4000000FFFF806B08B50368416B1A6822F4B3
:1014E40080621A60002242850A65816B0A6590F861
:1014F4003D1060294FF0200180F83D1080F83E2017
:1015040007D102641A6822F001021A60FFF749FB4E
:1015140008BD1A6822F001021A6001F0F7F808BD4C
:101524002DE9F341044618B9012002B0BDE8F08169
:101534000368DD0710D42368980758D423681A0772
:1015440000F19A8023685B0700F1B880A269002A41
:1015540040F019810020E8E7A64B9A6802F00C02DB
:10156400042A07D09A6802F00C02082A0AD15B68A0
:10157400590207D59F4B1B689A03DCD56368002B7F
:10158400D9D1D1E763689B4DB3F5803F11D12B6866
:1015940043F480332B60FFF7C9F9964D06462B6858
:1015A4009B03C8D4FFF7C2F9801B6428F7D9032032
:1015B400BBE7B3F5A02F04D12B6843F480232B6041
:1015C400E5E72A6822F480322A602A6822F480221D
:1015D4002A60002BDFD1FFF7A9F906462B689F0389
:1015E400A9D5FFF7A3F9801B6428F7D9DFE7814B5E
:1015F4009A6812F00C0F07D09A6802F00C02082ABD
:1016040011D15B685E020ED47A4B1A68950702D535
:10161400E268012A88D11A68216922F0F80242EAB4
:10162400C1021A608AE7E268734BB2B101221A6000
:10163400FFF77CF96F4D06462B68980707D52B6892
:10164400226923F0F80343EAC2032B6076E7FFF72D
:101654006DF9801B0228EFD9A9E71A60FFF766F934
:10166400644D06462B6899077FF568AFFFF75EF96E
:10167400801B0228F6D99AE76269604B7AB101228D
:101684001A60FFF753F95B4D06466B6F9F073FF5F2
:1016940059AFFFF74BF9801B0228F6D987E71A6088
:1016A400FFF744F9534D06466B6F98077FF54AAF31
:1016B400FFF73CF9801B0228F6D978E74D4B1A6CEA
:1016C40012F0805228D101921A6C42F080521A64AE
:1016D4001B6C03F080530193019B0126484D2B683A
:1016E400D9051BD5A368434D012B27D12B6F43F09C
:1016F40001032B67FFF71AF93E4D074641F288387C
:101704002B6F9B0739D5002E3FF420AF394A136C59
:1017140023F08053136419E70026DFE72B6843F4B2
:1017240080732B60FFF702F907462B68DA05D9D4DA
:10173400FFF7FCF8C01B0228F7D938E7052B04D1C2
:101744002B6F43F004032B67D0E72A6F22F00102CA
:101754002A672A6F22F004022A67002BCAD1FFF7F6
:10176400E5F841F2883807462B6F9807CBD5FFF789
:10177400DDF8C01B4045F7D919E7FFF7D7F8C01BC0
:101784004045BDD913E71B4DAB6803F00C03082B90
:101794003FF4CAAE1B4E0023022A336034D1FFF754
:1017A400C5F807462B6899011ED4226AE3691343DE
:1017B400626A43EA8213E26A43EA0263A26A0D4C54
:1017C4005208013A43EA02436B6001233360FFF796
:1017D400ADF8054623689A013FF5BCAEFFF7A6F8BD
:1017E400401B0228F6D9E2E6FFF7A0F8C01B022846
:1017F400D8D9DCE60038024000004742800E474258
:101804000070004060004742FFF790F804462B68E0
:101814009B017FF59FAEFFF789F8001B0228F6D9DC
:10182400C5E600BF134908B58B6803F00C03042B0D
:1018340003D0082B03D0104808BD104808BD4A68DF
:101844004B68496813F4800314BF0C480A48C1F379
:10185400881118BF002302F03F02A1FB0001FEF72C
:10186400CDFC044B5B68C3F3014301335B00B0FB65
:10187400F3F008BD003802400024F40000127A009E
:101884002DE9F0410D46044610B90120BDE8F08170
:10189400444B1A6802F00F028A4228D321688F074A
:1018A4002DD4C80740D43F4B1A6802F00F0295426A
:1018B40066D3226851076CD4130707D53A4A2169C5
:1018C400936823F4604343EAC1039360FFF7AAFFDC
:1018D400354B364A9B68C3F30313D35CD840344B6F
:1018E40018600020FEF7D8FF0020BDE8F081CAB2DE
:1018F4001A701B6803F00F039942C6D1CEE72A4B36
:1019040011F0040F1EBF9A6842F4E0529A600E0769
:1019140042BF9A6842F460429A609A68A06822F0D2
:10192400F00202439A60BCE762681F4B012A1DD192
:101934001B6813F4003FA8D01B4EB36823F00303C5
:101944001343B360FEF7F2FF41F288380746B368E9
:10195400626803F00C03B3EB820FA4D0FEF7E6FF3A
:10196400C01B4045F3D90320BDE8F081911E012935
:101974001B6802D813F0007FDDE713F0020FDAE7EB
:10198400EAB21A701B6803F00F039D427FF47DAF27
:101994008FE70549E0688B6823F4E05303438B60C9
:1019A4008AE700BF003C024000380240902D000846
:1019B40024000020036813F0050FF7B504463CD15A
:1019C40023689A0730D500230193444B444D1A6C85
:1019D40042F080521A641B6C03F080530193019B04
:1019E4002B6843F480732B60FEF7A0FF06462B6838
:1019F400D9054AD5394D2B6F13F440734BD1E368A5
:101A040003F44072B2F5407F344A63D1916823F005
:101A1400704021F4F81120F4407001439160116F7B
:101A2400C3F30B030B431367206810F008001FBFB8
:101A34002C4B227C1A60002025E02B4D274E0023DE
:101A44002B60FEF773FF074633681B0115D4A368A8
:101A540062681B0743EA8213C6F8843001232B60B3
:101A6400FEF764FF1D4D06462B681801A8D4FEF747
:101A74005DFF801B0228F7D904E0FEF757FFC01B67
:101A84000228E1D9032003B0F0BDFEF74FFF801B0D
:101A94000228ACD9F6E7E26802F440729342AED071
:101AA4002B6F124A0121116023F44073002111604D
:101AB4002B672B6FDA07A2D5FEF738FF41F2883780
:101AC40006462B6F9B079AD4FEF730FF801BB84263
:101AD400F7D9D7E7916821F4F8119FE7003802405D
:101AE40000700040E011474268004742400E474200
:101AF4000368DA68D20510B504460AD59B68D90490
:101B040007D500F0A9FC2268D368DBB263F4C07384
:101B1400D3602368DA6892050BD59B689B0408D5CB
:101B2400204600F00FF82268D368DBB263F4207318
:101B3400D360034B4FF400325A610123637710BD25
:101B4400003C01407047022310B580F83930036827
:101B5400196A41F211121142044608D1196A40F27D
:101B64004442114202BF1A6822F001021A60204660
:101B740000F0AAFA002084F8390084F8380010BD77
:101B840070477047704703681A69910710B5044697
:101B94000ED5DA6892070BD56FF002021A619B69C1
:101BA40001229B07027677D0FFF7EAFF0023237612
:101BB40023681A69500710D5DA6851070DD56FF0FC
:101BC40004021A619B69022213F4407F22762046A4
:101BD40068D0FFF7D5FF0023237623681A6912071C
:101BE4000FD5DA6810070CD56FF008021A61DB69AB
:101BF40004229907227620465AD0FFF7C1FF00231A
:101C0400237623681A69D20610D5DA68D0060DD572
:101C14006FF010021A61DB69082213F4407F227608
:101C240020464BD0FFF7ACFF0023237623681A69C4
:101C3400D10708D5DA68D20705D56FF001021A6119
:101C4400204600F0CCFC23681A69100608D5DA682F
:101C5400110605D56FF080021A61204600F0A4F841
:101C640023681A69520608D5DA68500605D56FF05C
:101C740040021A612046FFF785FF23681A6991061E
:101C840022D5DA6892061FD56FF0200220461A6129
:101C9400BDE8104000F087B800F098FC2046FFF73C
:101CA40070FF83E700F092FC2046FFF76AFF92E79B
:101CB40000F08CFC2046FFF764FFA0E700F086FCF0
:101CC4002046FFF75EFFAFE710BD036A10B501249D
:101CD4008C4023EA04030362036A8A401A430262C3
:101CE40010BD000010B5044600220068FFF7EDFFA8
:101CF4002368124A93420DD1196A41F2111211421A
:101D040008D1196A40F24442114202BF5A6C22F4CB
:101D140000425A64196A41F21112114208D1196A37
:101D240040F24442114202BF1A6822F001021A60D2
:101D3400012384F83930002010BD00BF00000140A9
:101D4400036A10B504248C4023EA04030362036A83
:101D54008A401A43026210BD10B50446002200688E
:101D6400FFF7EEFF2368196A41F21112114208D1FC
:101D7400196A40F24442114202BF5A6C22F40042F2
:101D84005A64196A41F21112114208D1196A40F2D7
:101D94004442114202BF1A6822F001021A60002074
:101DA40010BDFFF7D9BF704770470368DA6822F4A3
:101DB4009072DA605A6922F001025A61202380F895
:101DC4003A30704790F83930202B18D1A9B1A2B11C
:101DD40090F83830012B12D0C2840162828400232F
:101DE4000168C363212280F83920CA6880F838303A
:101DF40042F08002CA6018467047012070470220F2
:101E0400704790F83A30222B10B532D183680169BB
:101E14000268B3F5805F836A1FD15268C9B9C2F3FF
:101E2400080223F8022B8362C48D013CA4B2C4854A
:101E34006CB90368DA6822F49072DA605A6922F0A5
:101E440001025A61202380F83A3000F0D9FC0020C6
:101E540010BDD2B223F8012BE5E721B9591C526811
:101E640081621A70E0E75268591C816202F07F02B5
:101E7400F7E7022010BD000003681A68D96870B53E
:101E8400160704465D6907D196065AD58D0658D5BE
:101E9400BDE87040FFF7B5BF15F0010502D111F49C
:101EA400907F4ED0D30705D5CE0542BFE36B43F0F8
:101EB4000103E363500704D51DB1E36B43F0020350
:101EC400E363930704D51DB1E36B43F00403E363B9
:101ED400160704D51DB1E36B43F00803E363E36B1A
:101EE400002B66D0950604D5880602D52046FFF758
:101EF40088FF23685D69E26B1107204602D415F060
:101F040040051AD0FFF751FF23685A69520610D5CD
:101F14005A69606B22F040025A6150B1254B036547
:101F2400FEF789FD002844D0606BBDE87040036D66
:101F34001847204600F09EFC70BD00F09BFCE56352
:101F440070BD160627D50D0625D594F83920212A0B
:101F54002FD1A268B2F5805F226A17D11188C1F32C
:101F640008015960216979B902322262E28C013A8E
:101F740092B2E284EAB9DA6822F08002DA60DA68BE
:101F840042F04002DA6070BD0132EEE7511C21627A
:101F940012785A60EAE750060BD54A0609D5DA6882
:101FA40022F04002DA60202384F83930204600F021
:101FB4003BFC70BDBD1F000808B5806B0023C385C2
:101FC400C38400F057FC08BD90F8392090F83A001B
:101FD4001043704786B00023052853D8DFE800F08B
:101FE40003111E2B38450093274B28481A6B42F0E7
:101FF40001021A631B6B03F001030093009B06B0FC
:1020040070470193204B22481A6B42F002021A6374
:102014001B6B03F002030193019BF0E702931A4B3D
:102024001C481A6B42F004021A631B6B03F004038E
:102034000293029BE3E70393134B17481A6B42F096
:1020440008021A631B6B03F008030393039BD6E790
:1020540004930D4B11481A6B42F010021A631B6B68
:1020640003F010030493049BC9E70593064B0C4843
:102074001A6B42F080021A631B6B03F08003059312
:10208400059BBCE70020BAE700380240000002408C
:102094000004024000080240000C0240001002400C
:1020A400001C024008B5064900F0D0F9C0F3C43062
:1020B400023802289ABF034B185C002008BD00BFF9
:1020C400882A0008F42C000800F028BA30B5124918
:1020D40091B0054600F096F90190B8B12846FFF793
:1020E400E1FF1828044611D80C4BC340DB070DD57B
:1020F4000949284600F0AAF910F4801F214601A8D6
:1021040006D0FFF74EFE01A8FFF71DFD11B030BD4C
:10211400FFF7E8FDF7E700BF882A00081111000166
:10212400FEF704BC704708B5FEF7F4FBFEF77FFC2E
:10213400FFF7F8FF08BD08B5FEF7D2FBBDE808407D
:10214400FEF7FCB9064838B5A0F5A074A0F1140553
:102154001038FEF76BFBA5422846F7D138BD00BF07
:10216400880200200023012803F1010202D0400864
:102174001346F8E71421DBB24B43044A181D1044FC
:10218400816811B11A441369184770474801002047
:102194000120FEF763BC0220FEF760BC0420FEF7BA
:1021A4005DBC0820FEF75ABC1020FEF757BC38B5BA
:1021B40005242025A8B2FEF751FC013C4FEA450551
:1021C400F8D138BD38B506244FF48065A8B2FEF7BF
:1021D40045FC013C4FEA4505F8D138BD224B234963
:1021E40006221A7007221A75082283F82820092269
:1021F40083F83C200A2283F850201722002083F819
:10220400642083F8782083F88C2083F8A02083F856
:10221400B420282283F8C82083F8DC2083F8F02037
:1022240083F8042183F8182183F82C21D8601862DC
:1022340058639864D8651867C3F88400C3F8980095
:10224400C3F8AC00C3F8C000C3F8D400C3F8E80076
:10225400C3F8FC00C3F81001C3F82401C3F8380123
:10226400034A00F0C3BB00BF480100204921000815
:102274000000002030B5C36891FAA1F4B4FA84F4E4
:1022840091FAA1F10325B1FA81F1640005FA04F48D
:10229400490023EA040302FA01F11943C16030BD85
:1022A400431C04D00C3111F90C3C5A1C01D1002000
:1022B4007047984201F10C01F5D1012070470000EC
:1022C4002DE9F041474B00F00F08C0F3031401302F
:1022D4000E4601F0070753F8285003D14321424822
:1022E40000F0F5F82046FFF775FE0446826895FA7B
:1022F400A5F3B3FA83F395FAA5F103205B00B1FAD1
:1023040081F100FA03F322EA03034A0000FA02F21D
:102314001343A360874236D8DFE807F01D1D021D72
:10232400B8F1070FC6F3062017D9626A2B0A93FA8D
:10233400A3F1B1FA81F193FAA3F34FF00F0EB3FABC
:1023440083F389000EFA01F19B0022EA010200FAEC
:1023540003F3134363623B461AE0226A95FAA5F33A
:10236400B3FA83F395FAA5F14FF00F0EB1FA81F1A8
:102374009B000EFA03F3890022EA030200FA01F338
:1023840013432362E7E76A21174800F0A0F800230B
:10239400226895FAA5F0B0FA80F095FAA5F14FF00D
:1023A400030EB1FA81F140000EFA00F0490022EA6E
:1023B40000028B40013F1343012F236005D863685B
:1023C40032074CBF2B43AB436360C6F30112012AAF
:1023D40002D0022A18BF002229462046BDE8F04157
:1023E400FFF748BF502D0008F72C000891F9003082
:1023F4005A1C01D100207047834201D148687047BC
:102404000C31F3E7431C01D0FFF7F0BF0020704705
:102414004B6813B94FF0FF307047834202D191F9F2
:10242400000070470C31F3E708B1FFF7F1BF4FF03C
:10243400FF30704791F900305A1C01D1184670479B
:10244400834201D1886870470C31F3E7431C01D003
:10245400FFF7F0BF70470000034B1B6813B1034A3A
:1024640010681847704700BF88020020AC020020A3
:102474000148FFF73DBB00BF8C020020DFF834D0D9
:10248400002103E00C4B5B58435004310B480C4BC8
:1024940042189A42F6D30B4A02E0002342F8043B66
:1024A400094B9A42F9D300F013F800F0B3FAFEF79F
:1024B400E1F9704700800120182E00080000002078
:1024C400280000202800002010040020FEE7FEE77A
:1024D4000F49D1F8883043F47003C1F888300D4BAC
:1024E4001A68002042F001021A6098601A6822F00B
:1024F400847222F480321A60074A5A601A6822F4FD
:1025040080221A60D8604FF000638B60704700BF70
:1025140000ED00E000380240103000240368234A34
:1025240093420ED122494A6C22F001024A64214AA4
:10253400934217D102F57842536C23F480335364E9
:102544007047B3F1804F05D119490A6C22F001029A
:102554000A64ECE7184A93420DD115490A6C22F03B
:1025640002020A64154A93420DD102F57442536C77
:1025740023F40033E3E7124A93420DD10C490A6C69
:1025840022F004020A640F4A9342D9D102F5704240
:10259400536C23F48023D2E70B4A9342C7D102F54C
:1025A4000B32136C23F008031364704700000140DE
:1025B4000038024000400140000400400044014053
:1025C4000008004000480140000C0040436C2BB15F
:1025D400027E012A02D100210438184770470346BD
:1025E40004381B6C03B118477047000010B5064C43
:1025F400206808B1FFF7C7FA606A18B1BDE8104057
:10260400FFF7C1BA10BD00BFB0020020024B5868EA
:1026140008B1FFF7B8BA7047B0020020024B9868BF
:1026240008B1FFF7B0BA7047B0020020024BD86877
:1026340008B1FFF7A8BA7047B0020020024B18692E
:1026440008B1FFF7A0BA7047B0020020024B186A25
:1026540008B1FFF798BA7047B0020020024B986A9D
:1026640008B1FFF790BA7047B0020020C3689A42DD
:1026740010B504461CD171B9436E80F8581003B1EB
:10268400984794F8882004F1680120460823BDE89F
:102694001040FEF7EFB900230122C36580F85820EB
:1026A400C16D014402236831BDE81040FEF71EBA33
:1026B40010BD036E10B5044643B190F85820012AAA
:1026C40004D1C26D12B1C16D68309847022384F8F9
:1026D40058300023E3652046BDE81040FEF742BAB7
:1026E400C36D1F2BDEBFC36D0133C36590F8582043
:1026F400D2B2012A05D1C16D014402236831FEF72B
:10270400F5B97047002380F88830704790F8593045
:102714000BB9FEF727BA7047014B1868FEF7D6BA13
:1027240008030020014B1868FEF73ABE0803002096
:10273400014B5868FEF7CABA08030020014B5868D9
:10274400FEF72EBE08030020014B9868FEF7BEBAC0
:1027540008030020014B9868FEF722BE08030020FE
:1027640008B5074B90F8442053F82200FFF72CFCDF
:1027740000F02100A0F121035842584108BD00BFD8
:10278400B403002010B5044600B390F84430104A56
:1027940042F823100F4A002142F82300022290F944
:1027A4005A00FEF7DBF894F95A00FEF70BF9636E52
:1027B400B4F86A1094F8440013FA81F1064B01222C
:1027C40053F82000BDE81040FFF7FCBA10BD00BF6D
:1027D400640300208C030020B403002010B548B12A
:1027E4000649002351F82340A042DAB203D0013352
:1027F4000A2BF7D10A22104610BD00BFB4030020F3
:1028040010B5FFF7EBFF092808D8054B054A53F824
:10281400203052F82000BDE81040184710BD00BF1A
:10282400140300203C03002010B5FFF7D7FF09284C
:1028340018D80D4B53F820400C4B53F82030204649
:10284400984701300ED0636EB4F86A1094F84400CF
:1028540013FA81F1064B012253F82000BDE8104021
:10286400FFF7B0BA10BD00BF8C0300206403002042
:10287400B403002003681A68D20782B002D55B68EB
:10288400019308E01A689007F9D41A685107F6D43E
:102894001A681207F3D4019B02B0704708B52520CB
:1028A400FEF7B4F8024B1868BDE80840FFF7E4BA35
:1028B400B403002008B52620FEF7A8F8024B586898
:1028C400BDE80840FFF7D8BAB403002008B5472094
:1028D400FEF79CF8024B5869BDE80840FFF7CCBAF4
:1028E400B40300203A282DE9F041884633D8224B1E
:1028F4001C56621C2FD0C4F30315204E56F8253005
:1029040004F00F07FB40DB0710D51D492046FFF7F5
:10291400C7FC10B12046FFF7D9FB012303FA07F2E5
:1029240056F8253023EA020346F82530B8F1050F9E
:102934001DD8DFE808F003181214161A00212046E7
:10294400FFF7BEFC0F49012303FA07F251F82530C3
:10295400134341F82530BDE8F0811021EFE7202131
:10296400EDE70321EBE70121E9E70921E7E7462148
:102974000548FFF7ACFDE5E7912C0008DC030020D7
:10298400882A0008F4030020A02D00083A289ABFE2
:102994000B4B1B564FF0FF33C3F30312052A98BFAA
:1029A400084803F00F0398BF50F82220064888BF58
:1029B400002250F8233009B1936170471B04FBE7F0
:1029C400912C00080C000020502D0008FFF7A8BB34
:1029D40038B5044648B1FFF7A3FB0546FDF740FFB1
:1029E400FFF79EFB401B8442F8D838BD0B460146D6
:1029F400184600F001B8000010B5054C13462CB180
:102A04000A4601460220AFF3008010BD204610BDE7
:102A14000000000070B50D4E0D4CA41BA410002541
:102A2400A54209D10B4E0C4C00F020F8A41BA410B5
:102A34000025A54205D170BD56F8253098470135CB
:102A4400EEE756F8253098470135F2E7042E0008E2
:102A5400042E0008042E0008142E00080244034625
:102A6400934200D1704703F8011BF9E7F8B500BFA2
:102A7400F8BC08BC9E467047F8B500BFF8BC08BC5B
:042A84009E467047B3
:102A880000000000000C004012820000010000005D
:102A9800000C00401202010002000000000C00407F
:102AA8001282010003000000000C00401202020024
:102AB8000500000000000040128100000600000030
:102AC80000040040128200000700000000040040DB
:102AD80012020100080000000000014012810000FD
:102AE8000900000000000140120101000A00000076
:102AF80000000140128101000B00000000000140AD
:102B0800120102000F0000000000004012810000C6
:102B180010000000000400401282010011000000B3
:102B280000040040120202001300000000000040F0
:102B3800120101001400000000040040128200008D
:102B480015000000000400401202010016000000F9
:102B58000008004012820000170000000008004032
:102B68001202010018000000000800401282010053
:102B78001900000000080040120202001A000000BC
:102B880000000040128101001D000000000001400B
:102B9800128110001E000000000001401201110007
:102BA8001F000000000001401281110026000000F3
:102BB80000040040128200002700000000040040CA
:102BC80012020100280000000004004012820100E7
:102BD800290000000004004012020200FF0000006B
:102BE8000000000000000000030000000044004056
:102BF800120700000A000000001001401207000040
:102C0800FF000000000000000000000002000000BB
:102C180000440040120700001600000000100140A8
:102C280012070000FF000000000000000000000084
:102C38002F686F6D652F6A696D6D792F2E617264CB
:102C480075696E6F31352F7061636B616765732FBE
:102C580053544D33322F68617264776172652F73F4
:102C6800746D33322F312E352E302F7661726961B3
:102C78006E74732F434F534D494350492F766172F9
:102C880069616E742E6370700003020A1315141ABA
:102C98000809271607060519182A2CFF0D0E0F1705
:102CA8002D2E2F505122232B32292826250C0B1C80
:102CB8001B12111F1E1D24000104102120070622CB
:102CC80023251124000000000000000095060008DC
:102CD8007D070008410600086B0600085106000839
:102CE800D5060008D3070008FD07000804080C2FC4
:102CF800686F6D652F6A696D6D792F2E61726475C5
:102D0800696E6F31352F7061636B616765732F531F
:102D1800544D33322F68617264776172652F737412
:102D28006D33322F312E352E302F636F7265732F2E
:102D380061726475696E6F2F73746D33322F7069A9
:102D48006E6D61702E63000001000000020000003B
:102D5800040000000800000010000000200000002F
:102D68004000000080000000000100000002000098
:102D7800000400000008000000100000002000000F
:102D8800004000000080000000000000000000007B
:102D980001020304060708092F686F6D652F6A6929
:102DA8006D6D792F2E61726475696E6F31352F7074
:102DB80061636B616765732F53544D33322F6861BC
:102DC8007264776172652F73746D33322F312E35CB
:102DD8002E302F636F7265732F61726475696E6F21
:102DE8002F776972696E675F6469676974616C2EB1
:042DF8006300000074
:082DFC0034D4FF7F0100000048
:102E040069080008B90100086D070008E1210008FD
:042E1400950100081C
:102E18000000000001000000100000000000024057
:102E28000004024000080240000C0240001002406A
:082E3800001C02400024F4001C
:04000005080024814A
:00000001FF
